:020000040000FA
:020000000528D1
:080008005B2A831285018601C9
:1000100087018316D13081000B30850000308600C7
:10002000F030870005309F00831220308B00803035
:100030009F00A001A101A2010730A3000130A4008C
:100040000130A500B301A801A901AA01F030B40054
:100050008B1703302202031C2928AD01AE01AF012A
:10006000FE30A7002D30B6000630A9001A30AA00D5
:100070004D2199302D02031944281130AD0711305C
:10008000AE071130AF073228A201BA200030330288
:10009000031D53282030B600FE30A7001030200288
:1000A000031CA7138B2801303302031D5C28233067
:1000B000B600FD30A7008B2802303302031D6A28EA
:1000C000CD202D30B6003930A70010302E02031C91
:1000D000A7128B28EF302207031C4A28EA30220798
:1000E000031C5728DF302207031C4A28DA30220776
:1000F000031C6028BF302207031C4A28BA3022079D
:10010000031C5728AF302207031C4A28AA302207B5
:10011000031C60284A284D21B41B9428B30A0430DC
:1001200033020319B301AB28341B9828E720AB280E
:10013000341AAB2806302102031CA52855302102B1
:10014000031CAB288B139B22A6288B13A101A201B1
:10015000A901AA018B17A81C4528A921A8100130C4
:100160002502031D4528E62101302402031D4528F0
:10017000F821452881309F0046221F151F19BE28EF
:1001800075301E070318C92876301E02031CCB28C1
:100190000800281108002815080089309F00462211
:1001A0001F151F19D1281E08AC0083161E088312C4
:1001B000B700AB01B70DAC0DAB0DB1222F08AE00EF
:1001C000AE0E3008AE043108AF00AF0E08008B133E
:1001D0002330B600C030A7004D21341FF728341E4D
:1001E000F528B41AEA28F821EA282522EA2830302E
:1001F000A7004D21341F0429341E0229B41AF72800
:10020000E621F7281922F7280C30A7004D21341FCA
:100210001129341E0F29B41A0429A92104290922FD
:1002200004292030B600A901AA01A201F230A700DA
:100230004D21341F3129341E2729B41A18292030A2
:100240008400A522243020020318A00118292030A0
:1002500084003622F9302002031D18292330A00023
:1002600018294D21341F4A29341E4029B41A312936
:1002700021308400A522603021020318A101312918
:10028000213084003622F9302102031D31295930F2
:10029000A1003129B3018B17080036088400A71F7D
:1002A0005529000E8700803086009D21271F5E297A
:1002B0000008870040302718413086009D21840ABD
:1002C000A71E6829000E87002030A718223086005C
:1002D0009D21271E71290008870010302718113032
:1002E00086009D21840AA71D7929000E8700083009
:1002F00086009D21271D8029000887000430860084
:100300009D210708B400F030B405F0303402031D1D
:100310008B29B5019929B50A0130350203199C29A9
:100320003C303502031D97293230B5009C29F0304E
:10033000B400281C4D292810080041224122281908
:1003400086010230B8004B2286014122412241221F
:100350000800A50A2508A6000F30A6050A302602C7
:10036000031DB4290630A507BE21A60025082602D4
:10037000031CBB2908000130A5000800023024023C
:10038000031DD229003023020319CE292308A60019
:100390000330A605003026020319D0292830E529AC
:1003A0002930E529043024020319E4290630240207
:1003B0000319E429093024020319E4291130240225
:1003C0000319E4293130E52930300800A40A240853
:1003D000A6000F30A6050A302602031DF1290630BB
:1003E000A40713302402031C08000130A4000800F5
:1003F000A30A2308A6000F30A6050A302602031D13
:10040000032A0630A307A0302302031C0800A3011F
:100410000800A5030319162A2508A6000F30A60513
:100420002602031D08000630A5020800BE21A50013
:100430000800A403031D1E2A1230232A0F302402B1
:10044000031D08000930A4000800A303FF302302A5
:10045000031D2C2A6630342A2308A6000F30A60577
:100460002602031D08000630A302080080030008CE
:10047000B2000F30B2053202031D080006308002C0
:1004800008006930B800B80B432A08001630B800DD
:10049000B80B482A08000030B90000000000000036
:1004A000000000000000000000000000B90B4D2A11
:1004B000B80B4B2A0800F300030E8301F0000A0872
:1004C000F1008A010408F2000B1D7F2AAA0F692A95
:1004D000A90A38302A02031D722A01302902031D9D
:1004E000722A851235302A02031D7F2A0C30290218
:1004F000031C7F2AA901AA018B2285162814A0308B
:100500008B0083017208840071088A00700E8300DA
:10051000F30E730E090022308400A52260302202FF
:10052000031C0800A20121308400A52260302102B2
:10053000031C0800A10120308400A52224302002E1
:10054000031C0800A814A0010800800A0008B200DB
:100550000F30B2050A303202031D08000630800752
:1005600008002B0E0F39F03EAE00AE07E23EAF00A2
:10057000323EB1002B080F39AF07AF07B107E93E94
:10058000B000B007B0072C0E0F39B007B107B00D9F
:10059000B10DB109B10D2C080F39B107AE0D0730FF
:1005A000AD000A30B107B003031CD22AB007AF0375
:1005B000031CD62AAF07AE03031CDA2AAE07AD032D
:0605C000031CDE2A080006
:02400E00723FFF
:00000001FF
